:020000040800F2
:10000000983900209D010008BB0F00082D0F000843
:10001000B70F0008ED0C000867330008000000006F
:1000200000000000000000000000000005010008C2
:10003000F10C00080000000049010008C92900086F
:10004000B7010008B7010008B7010008B91D000892
:10005000B7010008B7010008B7010008B7010008A0
:10006000B7010008B7010008B7010008B701000890
:10007000B7010008B7010008B7010008B701000880
:10008000B7010008B7010008B7010008B701000870
:10009000B7010008B7010008B7010008B701000860
:1000A000B7010008B7010008B7010008B701000850
:1000B000952A0008B7010008152B0008B7010008B1
:1000C000B7010008B7010008B7010008B701000830
:1000D000B70100081D3000085D300008B7010008B6
:1000E000B7010008B7010008B7010008DFF810D019
:1000F00000F088FC00480047CF3F0008AFF30080C5
:1001000098390020224B19680868B0E8F00F80F396
:100110000988BFF36F8F4FF0000080F311884EF015
:100120000D0E70470000000006480068006880F36C
:10013000088862B661B6BFF34F8FBFF36F8F00DFE1
:1001400000BF00BF08ED00E0EFF30980BFF36F8F41
:100150000F4B1A6820E9F00F106008B54FF05000FF
:1001600080F31188BFF34F8FBFF36F8F05F016FA3E
:100170004FF0000080F31188BDE808401968086856
:10018000B0E8F00F80F30988BFF36F8F704700BFAE
:10019000F4000020EFF30580704700000648804718
:1001A00006480047FEE7FEE7FEE7FEE7FEE7FEE75C
:1001B000FEE7FEE7FEE7FEE7352A0008ED0000084F
:1001C00040EA01039B0703D009E008C9121F08C0D9
:1001D000042AFAD203E011F8013B00F8013B521E59
:1001E000F9D27047F0B480EA0102D40F4200B2EBBA
:1001F000410F02D20246084611464A0042D0C30DC2
:10020000DDB2C1F3C752AD1A202D35DAC1F31601A4
:1002100041F4000204B15242C5F1200602FA06F18F
:100220002A411044B3EBD05F23D0C4B1012DA0EB21
:10023000C35009DCF0BC4FF0004202EAC352DBB20B
:1002400000F5000000F03BBB400000F1807000EBC7
:10025000C350A0F1807040EAD170490009E049081C
:1002600041EAC071A0EBC35000F50000400800EB6C
:10027000C350F0BC00F01ABB6142012202EB410105
:10028000001BF6E7F0BC704781F00041AAE780F060
:100290000040A7E780EA010210B502F000434000E9
:1002A00022D04A001FD0010E01EB1261C0F35600AC
:1002B000C2F3560240F4000042F40002A0FB022008
:1002C00000047F39140400D0401C50EA124001D4CD
:1002D0004000491EC2B20C0604EBD010401C40087E
:1002E000802A02D003E0002010BD20F00100002988
:1002F00000DA0020184310BD30B480EA010202F099
:10030000004530F0004221F0004013D090B1C30D01
:10031000D40DC2F31601C0F31600E41A41F4000133
:1003200040F400027D34914201D3641C00E0490096
:10033000002C02DA30BC002070474FF4000000238C
:10034000914201D3891A034340084FEA4101F7D192
:1003500051B1914202D14FF0004105E002D24FF07D
:10036000010101E06FF0010103EBC450284430BCEF
:1003700000F09CBA2DE9FE4F804681EA0300C00FD1
:100380000C46009021F0004123F00045B8EB02003C
:10039000A94105D24046214690461C460B460246DE
:1003A00023F00040104347D0270DC7F30A00C3F3E2
:1003B0000A510290401A019040286BDAC3F31300EF
:1003C00040F4801B0098924620B10023D2EB030A30
:1003D00063EB0B0B01985946C0F14002504600F008
:1003E00034FA06460D4650465946019A00F04CFA3A
:1003F00010EB08006141002487EA115284EAE77398
:100400001A4340D0009A62B3019A012A4FEA075278
:1004100015DC001B61EB02014FF0004202EA0752BB
:10042000CDE90042001C41F5801132462B4600F018
:1004300083FA03B0BDE8F08F40462146F9E7001B80
:1004400061EB0201001C41F5801300185B4120188C
:10045000A2F5001747EB030140EAD570B6196D41CC
:1004600011E06D084FEA360645EAC0754FEA0752BB
:10047000001B61EB0201001C41F5801149084FEAA5
:1004800030000019514132462B4603B0BDE8F04F11
:1004900000F043BA0098012240000023D0EB020292
:1004A00063EBE073009821464FEAE074B8EB00007C
:1004B00061EB0401E9E783F000435BE781F0004171
:1004C00058E72DE9FE4F81EA030404F0004421F0CF
:1004D000004100944FF0000B23F0004350EA010468
:1004E0005ED052EA03045BD0C3F30A54C1F30A5549
:1004F0002C44A4F2F3340194A0FB0254C1F3130181
:1005000041F48011C3F3130343F4801301FB02444D
:1005100000FB034E840A970A44EA815447EA835752
:10052000A4FB076802958D0A05FB07854FEA932C0B
:1005300004FB0C542705029D4FEA065847EA16377C
:10054000B5EB08056EEB070C870E920E47EA811794
:1005500042EA8312A7FB0201B6EB0B0164EB000435
:100560002B0D43EA0C335E1844EB1C50DA4651461F
:10057000E7FB0201C5F313044FEA0B3343EA1453BC
:100580004FEA0432019C43EA0603A4F10C040294EE
:10059000009CCDE900B400F0CFF903B0BDE8F08FC6
:1005A00000200146F9E72DE9F04D81EA030404F04B
:1005B000004B21F0004514464FF0000A23F00041A3
:1005C00050EA050220D054EA01021DD0C5F30A57B3
:1005D0000246C5F31303C1F31300C1F30A5640F4F6
:1005E000801543F48013A7EB0608101BD64608F2CB
:1005F000FD3873EB050002D308F1010801E0921801
:100600005B41B8F1000F03DA00200146BDE8F08D30
:1006100000204FF48011064684460EE0171B73EB52
:10062000050705D3121B63EB050306434CEA010CD7
:1006300049084FEA300092185B4150EA0107EDD1BA
:1006400052EA030012D082EA040083EA050108435B
:1006500005D0101BAB4106D20122002306E0002288
:100660004FF0004302E06FF0010253101AEB060056
:100670004CEB085110EB0A0041EB0B01BDE8F04DCB
:1006800000F04BB9C10F80EAE0700844CA07962316
:10069000002100F014B90EB5C10F80EAE0700844E3
:1006A000CA07002140F233438DE80E000A460B468C
:1006B00000F042F903B000BD0EB540F233410291A3
:1006C0000021CDE900110A460B4600F035F903B0D0
:1006D00000BD20F00040C10DC0F3160040F4000042
:1006E0007F2901DA00207047962903DCC1F19601C9
:1006F000C8407047963988407047C1F30A5210B518
:10070000C1F3130140F2FF3341F480119A4201DA40
:10071000002010BD40F233439A42A2F2334203DC80
:10072000524200F0A1F810BD904010BD30B5041E3B
:1007300071F1000404DB4FF00044404264EB01011E
:10074000141E73F1000405DB1C464FF000435242B7
:1007500063EB0403994208BF904230BD01F00043AF
:1007600030B421F0004150EA010206D00A0DA2F592
:100770006072C1F31301002A02DC30BC0020704714
:10078000440F44EAC104C100E01830BC00EBC25081
:1007900000F08CB8002801DBC0F10040002901DB2B
:1007A000C1F1004181427047002801DBC0F10040E7
:1007B000002901DBC1F100418842704730B50B468A
:1007C000014600202022012409E021FA02F59D4281
:1007D00005D303FA02F5491B04FA02F52844151E55
:1007E000A2F10102F1DC30BD2DE9F05F05460020E9
:1007F00092469B4688460646814640241BE0284692
:1008000041464746224600F02FF853465A46C01A42
:10081000914110D311461846224600F016F82D1AC1
:1008200067EB01084F4622460120002100F00DF839
:1008300017EB00094E41201EA4F10104DFDC4846FD
:1008400031462A464346BDE8F09F202A04DB203A81
:1008500000FA02F1002070479140C2F1200320FA13
:1008600003F3194390407047202A04DB203A21FA11
:1008700002F00021704721FA02F3D040C2F12002B9
:100880009140084319467047202A06DBCB17203ACF
:1008900041FA02F043EAE07306E041FA02F3D04085
:1008A000C2F1200291400843194670470029A8BFB1
:1008B0007047401C490008BF20F00100704710B489
:1008C000B0FA80FC00FA0CF050EA010404BF10BC3E
:1008D000704749B1CCF1200421FA04F411FA0CF16B
:1008E00018BF012121430843A3EB0C01CB1D4FEAA4
:1008F00000614FEA102042BF002010BC704700EB9F
:10090000C35010440029A4BF10BC7047401C4900CC
:1009100008BF20F0010010BC704710B5141E73F121
:10092000000408DA401C41F1000192185B411A43AF
:1009300001D120F0010010BD2DE9F04D92469B46FB
:1009400011B1B1FA81F202E0B0FA80F220329046A1
:10095000FFF77BFF04460F4640EA0A0041EA0B011D
:1009600053465A46084313D0114653EA010019D0A2
:10097000C8F140025046FFF777FF05460E46504645
:1009800059464246FFF761FF084305D0012004E0C5
:1009900020463946BDE8F08D0020054346EAE07662
:1009A0002C4337430A986305E40AA0EB08000022B1
:1009B000FD0A44EA47540A3002D500200146E9E71F
:1009C000010510196941DDE9084500196941BDE8D3
:1009D000F04DA2E7C1F30A52C1F3130140F2FF3315
:1009E00041F480119A4202DA00200146704740F239
:1009F00033439A42A2F2334202DC5242FFF734BF41
:100A0000FFF723BF064C074D06E0E06840F0010306
:100A100094E8070098471034AC42F6D3FFF76AFB1E
:100A2000046600082466000870B58C1810F8015B95
:100A300015F0070301D110F8013B2A1106D110F877
:100A4000012B03E010F8016B01F8016B5B1EF9D17B
:100A50002B0705D40023521E0DD401F8013BFAE701
:100A600010F8013BCB1A921C03E013F8015B01F86C
:100A7000015B521EF9D5A142D8D3002070BD000001
:100A800070B5D378037013790B800B88022B08D1D3
:100A9000547903785B1E03EBC3035B00DB1C154D2D
:100AA000EC540B88032B08D1547903785B1E03EBBD
:100AB000C3035B001B1D0F4DEC540B88042B17DB8D
:100AC0000B88082B14DC55790B885B00DB1E04783F
:100AD000641E122606FB0433064CE55495790B88F8
:100AE0005B009B1E0478641E06FB0433014CE55436
:100AF00070BD00001C0000202DE9F04307ACF0CCD5
:100B000090F800C0ACF1010C0CEBCC0C4FEA4C0C93
:100B10000CF1030CDFF84C8118F80CC081F800C010
:100B200090F800C0ACF1010C0CEBCC0C4FEA4C0C73
:100B30000CF1040C18F80CC082F800C090F800C04A
:100B4000ACF1010C0CEBCC0C4FEA4C0C0CF1060C8C
:100B500018F80C8090F800C0ACF1010C0CEBCC0C38
:100B60004FEA4C0C0CF1050CDFF8F89019F80CC0AA
:100B700048EA0C2CA3F800C090F800C0ACF1010CBE
:100B80000CEBCC0C4FEA4C0C0CF1080CC84618F8D6
:100B90000C8090F800C0ACF1010C0CEBCC0C4FEACF
:100BA0004C0C0CF1070C19F80CC048EA0C2CA4F8FA
:100BB00000C090F800C0ACF1010C0CEBCC0C4FEA7B
:100BC0004C0C0CF10A0CC84618F80C8090F800C0C8
:100BD000ACF1010C0CEBCC0C4FEA4C0C0CF1090CF9
:100BE00019F80CC048EA0C2CA5F800C090F800C019
:100BF000ACF1010C0CEBCC0C4FEA4C0C0CF10C0CD6
:100C0000C84618F80C8090F800C0ACF1010C0CEB51
:100C1000CC0C4FEA4C0C0CF10B0C19F80CC048EA48
:100C20000C2CA6F800C090F800C0ACF1010C0CEB45
:100C3000CC0C4FEA4C0C0CF10E0CC84618F80C808A
:100C400090F800C0ACF1010C0CEBCC0C4FEA4C0C52
:100C50000CF10D0C19F80CC048EA0C2CA7F800C0D8
:100C6000BDE8F0831C00002010B5012000F042FC1C
:100C7000002000F03FFC10BD08B5014600200090A8
:100C8000034800900098084400900098008808BD30
:100C9000006C0040014908607047000000860D426A
:100CA00008B500220092044A0092009A0244009281
:100CB000009A116008BD0000006C004070B502464B
:100CC000CB781370042000BF0AE00D5C431E14783B
:100CD000641E122606FB0433034CE554431CD8B2B1
:100CE0001028F2DB70BD00001C00002000BFFEE7F2
:100CF00070472DE9F0410246002500260020002320
:100D00000024002791F803C00CF00F0591F803C0F0
:100D10000CF0100CBCF1000F03D091F802C04CEAAB
:100D2000050591F800C0BCF1000F31D01468002017
:100D30002BE04FF0010C0CFA00F3B1F800C00CEA04
:100D400003069E4220D183004FF00F0C0CFA03F7EC
:100D5000BC4305FA03FC4CEA040491F803C0BCF15F
:100D6000280F06D14FF0010C0CFA00FCC2F814C099
:100D70000AE091F803C0BCF1480F05D14FF0010C17
:100D80000CFA00FCC2F810C0401C0828D1D3146033
:100D9000B1F800C0BCF1FF0F34DD546800202EE034
:100DA00000F1080C4FF0010808FA0CF3B1F800C08C
:100DB0000CEA03069E4221D183004FF00F0C0CFA7F
:100DC00003F7BC4305FA03FC4CEA040491F803C0A2
:100DD000BCF1280F05D100F1080C08FA0CF8C2F894
:100DE000148091F803C0BCF1480F07D100F1080C42
:100DF0004FF0010808FA0CF8C2F81080401C0828CF
:100E0000CED35460BDE8F081416170470161704705
:100E100070B50C46FF2515701D700CE010F8015BD5
:100E2000167885EA06011D78064E765C75401570C9
:100E3000054D6D5C1D70251EA4F10106B4B2EDD107
:100E400070BD0000EC630008EC64000808B50121E7
:100E5000112000F02FFB012000F016FB002000F015
:100E6000FDFB0020FFF716FF4FF46040ADF80000D7
:100E700002208DF8020010208DF803006946064814
:100E8000FFF737FF002000F0FFFA4FF460410248FF
:100E9000FFF7BCFF08BD00000010014010B504467C
:100EA00001200D4908600D49C1F8B801204600F045
:100EB00017F800200849091F0860022003F01EF8F7
:100EC00001200649C1F8B801022003F017F80020FC
:100ED0000149091F086010BDBC01224200002242E6
:100EE00070B50446002500BF18E004F0800018B17A
:100EF00001200C49086002E000200A490860002037
:100F0000084908310860052002F0D8FF0120064991
:100F1000C1F8BC016006040E681CC5B2082DE4DBF4
:100F200070BD0000B40122420000224200BFFEE773
:100F30004CF6CC400149086070470000003000408A
:100F400010B500F001F810BD4AF6AA20014908606A
:100F500070470000003000400149486070470000C1
:100F600000300040014988607047000000300040B8
:100F70000149086070470000003000400146CA1770
:100F800001EB92729210A1EB820292B9642091FB64
:100F9000F0F200FB121050B94FF4C87091FBF0F260
:100FA00000FB121008B9012070470020FCE7012067
:100FB000FAE70020F8E700BFFEE7704770B50021B0
:100FC00000230F22C47804B3154C246804F4E064B1
:100FD000C4F5E064210AC1F10403CA40447804FA6C
:100FE00003F184781440214309010E4C0678A15581
:100FF000047804F01F050124AC4005786D11AD00A4
:1010000005F1E025C5F8004109E0047804F01F056A
:101010000124AC40044D0678761145F8264070BD99
:101020000CED00E000E400E080E100E00249014353
:10103000024A1160704700000000FA050CED00E064
:101040002DE9F0477A48806B7949C968884201DA0E
:10105000BDE8F087764A51681068FFF7A5FB07D214
:10106000734A51681068FFF70FF97149886106E00B
:101070006F4A11685068FFF707F96D4988616C4A3B
:1010800091699068FFF706F9694988620A46916993
:10109000106AFFF7A7F8664908620A46D1699069A5
:1010A000FFF7F2F807466248016A62480068FFF7F6
:1010B000F1F85F49486239465F480068FFF7EAF88F
:1010C0005B49C862C86A0021FFF764FB06D2584832
:1010D000C16A0020FFF7D8F85549C8625448846AAD
:1010E0000146C86BFFF7CEFA05462146FFF752FBD3
:1010F00006D24F49C86BFFF7C5FA4D4948630BE06C
:1011000000212046FFF746FB04D84948006B4849B8
:10111000486301E046484463454880694449C861E2
:101120000020886348684FF07E51FFF75BF8054662
:101130003F4801682846FFF72DFB12D200213F48A7
:1011400001F0CDFE3E49097841F004013C4A11709E
:101150000846FFF7A3FE02203A49087000203449F0
:101160004862334A11685068FFF71EFB29D23449A0
:10117000097801F0FB01324A11700846FFF78EFE34
:101180002B49C86BFFF77EFA80462949486B2E49E8
:10119000FFF780F881464146FFF7AEF806464FF06C
:1011A0007E51FFF771F80546FFF793FA274908606B
:1011B0000846008881B2214801F091FE01202149B2
:1011C000087020480078012816D121480088C01EE8
:1011D0002049096888420FDB0021184801F07FFE92
:1011E0001749097801F0FB01154A11700846FFF70D
:1011F00055FE00201349087012480078022815D1C6
:10120000144800681249098888420FDB00210B4806
:1012100001F065FE0A49097801F0FB01084A1170E6
:101220000846FFF73BFE00200649087000BF0FE7A5
:101230006C070020CC000020D000002000040040FB
:101240007C050020840500200000C843D400002055
:101250008C050020A40500200648074988604FF44B
:10126000FA70C860C820C8634FF07E500863002041
:10127000886370470000DC426C07002030B589B0FD
:1012800005460C460121C80200F014F90121042092
:1012900000F010F918208DF823004FF48070ADF89D
:1012A000200003208DF8220008A91B48FFF721FD2C
:1012B0000020ADF81A00ADF81600ADF81850ADF8E2
:1012C00014408DF81C0005A9144801F00DFE01A87A
:1012D00001F0F7FD6020ADF804000020ADF80C002F
:1012E0000120ADF806000020ADF80A0001A90B4866
:1012F00001F0A4FC0121094801F077FC082107480E
:1013000001F0E8FC0121054801F054FC01210348EB
:1013100001F05FFC09B030BD00080140002C014025
:1013200030B589B005460C460121C80200F0C2F86C
:101330000121042000F0BEF818208DF823004FF49E
:101340000060ADF8200003208DF8220008A91B489A
:10135000FFF7CFFC0020ADF81A00ADF81600ADF88D
:101360001850ADF814408DF81C0005A9144801F080
:10137000BBFD01A801F0A5FD6020ADF80400002030
:10138000ADF80C000120ADF806000020ADF80A0011
:1013900001A90B4801F04AFD0121094801F025FC93
:1013A0000821074801F080FD0121054801F002FCF9
:1013B0000121034801F00DFC09B030BD00080140D7
:1013C000002C014030B589B005460C460121084685
:1013D00000F060F80121042000F06CF818208DF86E
:1013E00023000220ADF8200003208DF8220008A978
:1013F0001648FFF77EFC0020ADF81A00ADF8160085
:10140000ADF81850ADF814408DF81C0005A94FF048
:10141000804001F069FD01A801F053FD6020ADF8A6
:1014200004000020ADF80C000120ADF806000020FB
:10143000ADF80A0001A94FF0804001F055FC0121F0
:10144000880701F0C6FB09B030BD0000000801406C
:1014500010B504462146024801F03DFD10BD0000D4
:10146000002C014010B5044621464FF0804001F0A9
:1014700034FD10BD10B504462146024801F031FD8F
:1014800010BD0000002C01400149086270470000B7
:1014900000000E4229B1064AD2690243044BDA61C8
:1014A00004E0034AD2698243014BDA6170470000CD
:1014B0000010024029B1064A92690243044B9A6126
:1014C00004E0034A92698243014B9A61704700002D
:1014D0000010024029B1064AD2680243044BDA6088
:1014E00004E0034AD2688243014BDA60704700008F
:1014F0000010024001490860704700004004424269
:1015000030B500210022002400232D4D6D6805F028
:101510000C0121B1042905D0082923D105E0294D6A
:10152000056022E0274D05601FE0254D6D6805F43C
:101530007012234D6D6805F48034022505EB92424C
:101540001CB9214D554305600BE01D4D6D6805F438
:1015500000351DB11C4D5543056002E0194D554342
:10156000056002E0174D056000BF00BF144D6D68B7
:1015700005F0F0010909154D6B5C0568DD4045601B
:101580000F4D6D6805F4E061090A104D6B5C45680C
:10159000DD4085600A4D6D6805F46051C90A0B4D48
:1015A0006B5C4568DD40C560054D6D6805F44041E4
:1015B000890B074D6B5CC568B5FBF3F5056130BD64
:1015C0000010024000127A0000093D00DE000020F9
:1015D000EE00002010B501460022002300204A1131
:1015E000012A02D1094C236806E0022A02D1074CE5
:1015F000236A01E0054C636A01F01F020124944054
:101600001C400CB1012000E0002010BD0010024081
:101610001149096821F480310F4A116011460968A7
:1016200021F480211160B0F5803F03D0B0F5802F08
:101630000ED106E00849096841F48031064A11607C
:1016400007E00549096841F4A021034A116000E060
:1016500000BF00BF704700000010024000210B4A8D
:1016600011700A4A203A82F82010012802D004287A
:1016700008D103E00121054A117004E00521034A65
:10168000117000E000BF00BF704700002010024052
:1016900001490860704700003C0442420249096A5F
:1016A0000143014A116270470010024010B586B034
:1016B000044600F057FD20213348FFF7A5FB4021E9
:1016C0003148FFF7A3FB01210C20FFF7F3FE0121B6
:1016D0008803FFF7EFFE4FF40060ADF81400102010
:1016E0008DF8170003208DF8160005A92648FFF78E
:1016F00000FB4FF40070ADF8140018208DF81700AF
:1017000005A92248FFF7F5FA4FF48060ADF8140000
:1017100004208DF8170005A91C48FFF7EAFA0121FB
:101720008803FFF7D7FE00214FF48040FFF7D2FE79
:1017300001940020ADF80800ADF80A00ADF80C00E7
:10174000ADF810000C20ADF80E0001A9104801F012
:1017500095FD25208DF8000000208DF80100012066
:101760008DF803006846FFF729FC012240F225515D
:10177000074801F05EFD0121054801F017FD00203A
:101780000449086006B010BD000C0140000801408B
:1017900000380140AC81214270B505460E4601205B
:1017A0000E49086000240CE000BF40210C4801F005
:1017B00009FD0028F9D0295D094801F0D0FD601C21
:1017C000C4B2B442F0DB00BF4021054801F0FAFC8E
:1017D0000028F9D000200149086070BDAC81214289
:1017E0000038014010B5EE20B4490870B5204870AB
:1017F00005208870FF204876FC208876FF20C87678
:1018000008770120AE490860AE480068B0F5FA7F5D
:1018100007DCAD48C078AD490870AB480079AC49E9
:101820000870AC480068B0F57A7F07DCA6484079BC
:10183000A9490870A4488079A8490870A34800788D
:101840009E49C870A24800780871A3480078487182
:10185000A24800788871A2480078401E00EBC000C2
:1018600040000A309F49095C9D480078401E00EB0B
:10187000C000400009309B4A105C41EA00209A49B0
:10188000088097480078401E00EBC00040000C30F4
:101890001146095C92480078401E00EBC0004000F1
:1018A0000B30105C41EA0020904908808C48007899
:1018B000401E00EBC00040000E301146095C884815
:1018C0000078401E00EBC00040000D30105C41EA83
:1018D00000208749088084480088B0F57A7F15DCAD
:1018E0007F480078401E00EBC000400009301146E0
:1018F000085C804908707A480078401E00EBC00000
:1019000040000A301146085C7B490870774800881F
:10191000B0F57A7F15DC72480078401E00EBC000FD
:1019200040000B306F49085C744908706C480078BF
:10193000401E00EBC00040000C306A49085C704952
:1019400008706B480088B0F57A7F15DC6448007831
:10195000401E00EBC00040000D306249085C694940
:1019600008705F480078401E00EBC00040000E3059
:101970005C49085C644908705E4800784F49C8714A
:101980005D48007808725D48007848725C480078CD
:1019900088725C480078C8725B48007808735B48BE
:1019A000006841F28831884207DC4748C07C5849CA
:1019B00008704548007D57490870554800783F49F0
:1019C00048735448007888734548007807283CDA03
:1019D00043480078401E00EBC0004000C01C414955
:1019E000085C182831DA3E480078401E00EBC00041
:1019F0004000001D085C3C2827DA4748007818287A
:101A000023DA464800783C281FDA354800782B490D
:101A1000C87333480078401E00EBC0004000C01C73
:101A20003049085C254908742D480078401E00EBB9
:101A3000C0004000001D2B49085C2049487436480E
:101A40000078887435480078C874354800781B4998
:101A5000087534480078487533480078887517232E
:101A60000322324802F01DFA314B324A14212F482A
:101A7000FFF7CEF92F4800781049C8752C48007838
:101A8000087600240DE000BF40212B4801F09AFBAE
:101A90000028F9D00948015D274801F060FC601C6E
:101AA000C4B21D2CEFDB00BF4021234801F08AFBAC
:101AB0000028F9D000200249086010BD88000020ED
:101AC000AC812142A40500200C340020A500002098
:101AD000A6000020A8050020A7000020A8000020E4
:101AE0008B0500201C000020AC000020B00000206E
:101AF000AE000020B2000020B3000020B60000209D
:101B0000B7000020B4000020B5000020AC05002084
:101B1000A9000020AA0000208205002083050020E3
:101B2000840500208505002086050020CC060020C5
:101B3000B9000020B8000020003801401CB519A1F0
:101B400003C9CDE900010120184908601848007850
:101B50008DF8030016480078401C154908700846A7
:101B60000078062801DD0120087000240DE000BF88
:101B70004021104801F026FB0028F9D01DF8041080
:101B80000C4801F0ECFB601CC4B2082CEFDB00BF7A
:101B90004021084801F016FB0028F9D00020034935
:101BA00008601CBDEEB50100FFFCFFFFAC812142C7
:101BB0007D05002000380140024909888143014A1F
:101BC00011807047042800400348008840F010004E
:101BD000014908807047000004280040034800883D
:101BE0004FF6EF7108400149088070470428004013
:101BF0002DE9F04106460F464FF00008002400256D
:101C000000F082F880463C48B8FBF0F43B4800887E
:101C1000A0423CD039490C8040F2B27510E0284611
:101C2000FFF7ACF940B1B4F5B77F02D3A4F5B774B0
:101C300004E0681C85B206E0A4F26D14681C85B24D
:101C4000B4F5B67FEBD800BF2D488580002516E09F
:101C50002B498888FFF792F930B1012D04D11D2C52
:101C600001D31D3C09E00CE02648405DA04203D8AA
:101C70002448405D241A00E003E0681C85B21C2C57
:101C8000E6D200BF681C1E498871601CC8711A48E2
:101C9000B8FBF0F100FB11844FF46160B4FBF0F08D
:101CA000174908704FF46160B4FBF0F100FB11407C
:101CB0003C21B0FBF1F0124948704FF46160B4FB75
:101CC000F0F100FB11403C21B0FBF1F201FB1200EE
:101CD0000B4988700B46DA799979988800F030F8CA
:101CE0000749087208460078307008464078387016
:101CF0000020BDE8F081000080510100BE000020FE
:101D000060070020F8650008002103480188001FD3
:101D1000008841EA004070471C280040014600202E
:101D2000064A12880A40D0B2044A121F12880A409A
:101D300012B108B1012000E00020704704280040E3
:101D4000F0B503460C461546642093FBF0F0C6B28E
:101D5000642093FBF0F700FB1730C1B2132E02DDB5
:101D600001F16400C1B20846CF1701EB977701EB90
:101D7000A707BAB2072092FBF0F700FB172082B248
:101D80005719601EDFF82CC01CF80000384482B2DE
:101D9000CF1701EB9777BF10A1EB87071FB9032C73
:101DA00001DA501E82B2072092FBF0F700FB1720E9
:101DB000C0B2F0BDEC65000810B50120FFF7AEFF22
:101DC00018B10A490A48FFF713FF0220FFF7A6FFE0
:101DD00030B10220FFF7F0FE04490548FFF708FF85
:101DE0000520FFF7E9FE00F00BF910BDBD00002053
:101DF000BC00002029B1064A12880243044B1A8015
:101E000004E0034A12888243014B1A8070470000A5
:101E1000002800401CB5002401214FF0C050FFF7FE
:101E200039FB0120FFF730FB0420FEF725FF45F2C8
:101E30005001884240D0FEF717FF4FF48030FFF783
:101E4000E7FB04E0601CC4B20A2002F037F831203E
:101E5000FFF7C0FB08B9FA2CF4DBFA2C01DB0120F8
:101E60001CBD4FF44070FFF719FC0120FFF710FC78
:101E700000F0C6F800F0CEF801210846FFF7BAFFDF
:101E800000F0BEF8FFF7A0FE4FF2244000F0A8F8E3
:101E900000F0B6F8002000900346012209210190CD
:101EA00040F2E77000F02AF8FFF798FE45F2500183
:101EB0000420FEF7F5FE07E000F0ACF8012108462B
:101EC000FFF798FF00F09CF800F00AF80249034879
:101ED000FFF78EFE0020C3E7BD000020BC000020FD
:101EE00008B503208DF8000001208DF801008DF861
:101EF00003006846FFF762F808BD00002DE9F05FB7
:101F000006460F4690469946DDE90AAB002440F2AA
:101F1000B270864203DB40F63300864202DD0120C8
:101F2000BDE8F09F40F2B2750AE02846FFF726F8B8
:101F300010B12048044401E01F480444681C85B2E5
:101F4000B542F2DB781EC7B2002510E01B48405DA9
:101F500040F2A321484304EBC0143046FFF70EF8CB
:101F600018B1012D01D116480444681C85B2BD4248
:101F7000ECDBA8F1010040F2A321484304EBC014BC
:101F8000C9EB4910C0EB092004EB0014CAEB0A109E
:101F900004EB80045C4401214FF0C050FFF77AFA53
:101FA0000120FFF771FA204600F00CF800F028F845
:101FB0000020B5E70085E2018033E101F865000803
:101FC0008051010000B50246FFF7FEFD100C0349E9
:101FD0000880091D0A80FFF701FE00BD1828004097
:101FE00000B50246FFF7F0FDC2F303400349088045
:101FF000091D0A80FFF7F2FD00BD0000082800401F
:1020000000BF0348008800F020000028F9D0704786
:1020100004280040074800884FF6F771084005493A
:10202000088000BF0348008800F008000028F9D0AD
:1020300070470000042800402DE9FC4705460E4685
:1020400017469846DDE90A9A002401214FF0C05056
:10205000FFF720FA0120FFF717FAFEF705FE4FF40D
:102060008030FFF7D5FA04E0601CC4B20A2001F00A
:1020700025FF3120FFF7AEFA08B9FA2CF4DBFA2C71
:1020800002DB0120BDE8FC874FF44070FFF706FB40
:102090000120FFF7FDFAFFF7B3FFFFF7BBFF0121B8
:1020A0000846FFF7A7FEFFF7ABFFFFF78DFD4FF2E6
:1020B0002440FFF795FFFFF7A3FF43463A4631461A
:1020C0002846CDE9009AFFF719FFFFF787FD45F293
:1020D00050010420FEF7E4FDFFF702FF0249034828
:1020E000FFF786FD0020CDE7BD000020BC000020EA
:1020F00010B502460020104604E04318084CE35C8B
:102100002354401CC1F180038342F6DCC1F18000FE
:1021100003E00023024C2354401C8028F9DB10BD4F
:102120000C34002010B501F045F96C22002109485B
:1021300001F068F96D2300220649074801F0B1FE5D
:1021400001226D21054801F05DF904480078044939
:10215000087010BDF40500201C00002016000020AF
:102160008B05002008B501210820FFF7A3F9E02026
:10217000ADF8000010208DF8030003208DF8020058
:1021800069460448FEF7B5FD80210248FEF73CFE93
:1021900008BD0000000C014000B587B001210420FB
:1021A000FFF788F901210803FFF784F9E020ADF873
:1021B000180018208DF81B0003208DF81A0006A9BE
:1021C0001748FEF796FDE0211548FEF71FFE002098
:1021D000ADF804004FF48270ADF806000020ADF8B1
:1021E00008000220ADF80A000120ADF80C00400202
:1021F000ADF80E003820ADF810000020ADF8120048
:102200000720ADF8140001A9064800F067F8012185
:10221000044800F049F8FF2000F006F807B000BDC0
:10222000000801400030014070B50546002405E07B
:10223000601CC4B2C82C01DD002070BD02210E4814
:1022400000F03EF80028F3D029460B4800F044F88F
:10225000002405E0601CC4B2C82C01DD0020ECE7BE
:102260000121054800F02CF80028F3D0024800F0C6
:1022700030F8C0B2E1E700000030014010B504467C
:10228000074800884FF6C77108400549088008468E
:102290000088204308800121024800F005F810BDA5
:1022A000003800400030014021B1028842F0400275
:1022B000028004E002884FF6BF731A400280704724
:1022C0000246002013890B400BB1012000E00020E2
:1022D00070470146888970478181704710B5002298
:1022E000028802F441520B884C8823438C88234394
:1022F000CC8823430C8923434C8923438C89234373
:10230000CC8923431A430280838B4FF2FF7423400E
:1023100083830B8A038210BD1FB5BBE202F026FD4A
:10232000FA490870FA48FB49FB4AFC4BCDE90032F8
:10233000CDE90210FA4BFB4AFB49F448FEF7DCFBFF
:102340000821FA48FFF728FAC82001F0FBFDFFF743
:10235000F5FBC82001F0F6FD80230022F449F54882
:1023600001F09FFD0020F449087031E2F148007847
:1023700001287DD1EF4840780328FAD1ED48C07894
:10238000EE490860EB480079096840EA0120EB4912
:102390000860E8484079EA490860E64880790968B9
:1023A00040EA0120E6490860E248C07CE54908604F
:1023B000E048007D096840EA0120E2490860D84809
:1023C00000881438DD490968884214DCDB4801685C
:1023D000D3480088143081420DDCD048008864382E
:1023E000D7490968884206DCD5480168CB4800888F
:1023F0006430814212DDD448008840F26221884274
:102400000CDDD249097841F00101D04A117008462B
:10241000FEF744FD0120CE4908700BE0CB49097856
:1024200001F0FE01C94A11700846FEF737FD002091
:10243000C7490870C1480068B0F5167F3EDABF484A
:10244000006810F11E0F39DDC2480068BB490968F9
:10245000401AC149086008460068002803DA0846A7
:10246000006840420860BC480068032804DB00E0C4
:102470008FE0B848006808BBA9480088FEF71CF93F
:1024800006460022B54BFEF78EF80446FEF766F9C5
:10249000B3490860A9480068FEF7FDF80646002227
:1024A000AE4BFEF780F80446FEF758F9AC49486099
:1024B000FEF7C6FDA1480068A6490860A04801686B
:1024C000964800883230814214DDA049097841F0F5
:1024D00008019E4A11700846FEF7E0FC9B49097806
:1024E00001F0EF01994A11700846FEF7D7FC012070
:1024F0009C490870894800883238914909688842A7
:1025000014DD9249097841F01001904A1170084693
:10251000FEF7C4FC8D49097801F0F7018B4A117070
:102520000846FEF7BBFC02208E4908708D480078F3
:10253000012811D1824800687849098888420BDC5B
:102540008249097801F0E701804A11700846FEF7D8
:10255000A5FC00208349087082480078022811D128
:10256000774800686D49098888420BDB774909780C
:1025700001F0E701754A11700846FEF78FFC002054
:1025800078490870FFF72EF917210020FFF7B0FDFA
:102590001EE168480078EE2821D166484078B628C8
:1025A0001DD164488078032819D1624A6E496F486A
:1025B000FEF766FA56485749574A584BCDE900325C
:1025C000CDE90210564B574A57495048FEF794FA46
:1025D00000F0E2FF0B210020FFF78AFDF8E05548EC
:1025E0000078EE2824D153484078B62820D15148AD
:1025F000807804281CD14F48C0785D4908700020BD
:102600000090034601220921019040F2E770FFF794
:1026100013FD574800783D490870554800785549E2
:10262000087000F0B9FF08210020FFF761FDCFE03E
:1026300040480078EE281ED13E484078B6281AD18E
:102640003C488078012816D13A494848FEF736FBC5
:102650002F483049304A314BCDE90032CDE90210E4
:102660002F4B304A30492948FEF746FA1421002002
:10267000FFF73EFDACE02F480078EE2814D12D483E
:102680004078B12810D12B48807811280CD12948E6
:10269000C07BFF2808D12648007CFF2804D11121E7
:1026A0000020FFF725FD93E022480078EE2814D1A2
:1026B00020484078B12810D11E48807811280CD1CC
:1026C0001C48807BFF2808D11948C07BFF2804D113
:1026D00010210020FFF70CFD7AE016480078EE2864
:1026E0004AD114484078B12846D112488078112840
:1026F00042D11048007BFF283ED10D48407BFF2887
:102700003AD10E210020FFF7F3FC61E08B05002099
:102710009405002092050020900500208E050020E1
:102720008C05002097050020960500209B050020C1
:10273000E00600200C340020BA000020A405002090
:10274000A8050020AC050020880500207C0500209D
:1027500086050020B40500207805002000002440F4
:102760006C07002085050020800500207E050020E4
:10277000980500207605002047480078EE2814D1FF
:1027800045484078B12810D14348807801280CD1C1
:102790004148C079FF2808D13F48007AFF2804D17A
:1027A00009210020FFF7A4FC12E000243A48007839
:1027B00018B101210020FFF79BFC00E0641C3648A3
:1027C000005D0028FAD0E1B20020FFF791FC00BFC5
:1027D0008021314801F0DCFB00283FF4C7AD2F48D1
:1027E0000088B0F57A7F52DC2D480088B0F57A7FFA
:1027F0004DDC2A480088FDF75FFF80460022294B08
:10280000FDF7D1FE06460022274BFDF75AFE824611
:102810000022264BFDF7AEFD0446FDF76EFF80B2A9
:102820000390FEF715FE1E480088FDF745FF06469B
:1028300000221C4BFDF7B7FE804600221A4BFDF725
:1028400040FE82460022194BFDF794FD0446FDF739
:1028500054FF80B20390FEF705FE15480088FDF78F
:102860002BFF804600220F4BFDF79DFE06460022FF
:102870000D4BFDF726FE044600220C4BFDF77AFDBA
:102880008246FDF73AFF80B20390FEF7F3FD002089
:102890000849087042E500000C3400209005002033
:1028A000920500200000594000000C4000003C4010
:1028B00094050020BA00002010B500F001F810BD0A
:1028C0000CB50020019000903348006840F480303F
:1028D0003149086000BF3048006800F400300090C3
:1028E0000198401C0190009818B90198B0F5A06FAC
:1028F000F1D12948006800F4003010B101200090A7
:1029000001E0002000900098012843D1234800688E
:1029100040F01000214908600846006820F00300DC
:1029200008600846006840F0020008601A484068E5
:10293000194948600846406848600846406840F4C5
:10294000806048600846406820F47C104860084673
:10295000406840F4E81048600846006840F0807025
:10296000086000BF0C48006800F000700028F9D033
:102970000948406820F0030007494860084640685D
:1029800040F00200486000BF0348406800F00C00BF
:102990000828F9D10CBD00000010024000200240C0
:1029A000042808D14FF0E021096941F004014FF0FB
:1029B000E022116107E04FF0E021096921F00401F4
:1029C0004FF0E0221161704710B503F069FA012859
:1029D00001D002F087FE10BD70B505460420FFF758
:1029E000DFFF104800681049B0FBF1F00F49087094
:1029F0000C4800680C49B0FBF1F44FF47A70444382
:102A000001200B4908804FF0E020006940F00200EF
:102A10004FF0E021086108464461006940F0010080
:102A2000086170BD0000002040420F00D800002067
:102A3000DA00002010B51348006840F00100114989
:102A4000086008464068104908400E49486008463A
:102A500000680E4908400B4908600846006820F4E9
:102A6000802008600846406820F4FE0048604FF46B
:102A70001F008860FFF720FF4FF0006004490860E6
:102A800010BD0000001002400000FFF8FFFFF6FE3E
:102A900008ED00E010B50121880700F0B5F840B15D
:102AA0000448806B401C034988630121880700F0BB
:102AB0008DF810BD6C0700201FB501210846FEF7F8
:102AC000E9FC1C208DF80C0003208DF80D0001207E
:102AD0008DF80F0003A8FEF771FA4FF47A70ADF885
:102AE00004004720ADF800000020ADF80200694660
:102AF0004FF0804000F0F8F901221146900700F0F5
:102B000094F80121880700F061F80121880700F09E
:102B100060F81FBD10B501210D4800F075F8B0B187
:102B200001210B4800F052F80A480088401C09496E
:102B3000088009480078401C07490870084600785A
:102B4000052804DDFEF7FCF900200349087010BDDC
:102B500000080040880500208A0500207FB5054652
:102B60000C4601210420FEF795FCADF80850ADF8A5
:102B700004400020ADF80A00ADF8060001A90C4899
:102B800000F0B2F901221146094800F04EF81E206B
:102B90008DF8000002208DF8010001208DF803005F
:102BA0006846FEF70BFA0121014800F012F87FBDDC
:102BB0000008004021B1028842F08002028004E057
:102BC00002884FF67F731A4002807047CA43028220
:102BD000704721B1028842F00102028004E00288BD
:102BE0004FF6FE731A400280704731B1B0F84420AE
:102BF00042F40042A0F8442005E0B0F84420C2F3BB
:102C00000E02A0F84420704730B502460020002391
:102C10000024158A05EA0103958905EA010413B128
:102C20000CB1012000E0002030BD1AB183890B43B4
:102C3000838102E083898B438381704770B50024D0
:102C400000220023058C4FF6FE7635400584028C69
:102C50008388048B4FF68F752C40B51E2C400D8851
:102C60002C43751E2A400D892A434D882A43144D52
:102C7000A8420BD0134DA84208D0134DA84205D04E
:102C8000124DA84202D0124DA84213D14FF6F7754B
:102C90002A404D892A434FF6FB752A408D882A43E6
:102CA0004FF6FF652B404FF6FF552B408D892B4388
:102CB000CD892B4383800483CD888586028470BDB3
:102CC000002C01400034014000400140004401401C
:102CD000004801400A460021018B4FF6F773194066
:102CE000114301837047000070B5002400220023C7
:102CF000058C4FF6EF7635400584028C8388048B73
:102D000048F6FF752C404FF6FF452C400D884FF6D6
:102D1000FF7606EA05252C434FF6DF752A400D891C
:102D200006EA05152A434D8806EA05152A43154D7E
:102D3000A84202D0144DA8421DD14FF67F752A40FB
:102D40004D894FF6FF7606EA05152A434FF6BF7503
:102D50002A408D8806EA05152A434FF6FF352B4099
:102D60004FF2FF752B408D8906EA85052B43CD89EF
:102D700006EA85052B4383800483CD88058702847A
:102D800070BD0000002C01400034014070B50024EB
:102D900000220023058C4FF6FF6635400584028C27
:102DA0008388848B4FF68F752C404FF6FC752C4032
:102DB0000D882C434FF6FF552A400D894FF6FF76BC
:102DC00006EA05252A434D8806EA05252A43154DBE
:102DD000A84202D0144DA8421DD14FF2FF752A40DF
:102DE0004D894FF6FF7606EA05252A434FF6FF3553
:102DF0002A408D8806EA05252A434EF6FF752B40AA
:102E00004DF6FF752B408D8906EA05152B43CD89BC
:102E100006EA05152B4383808483CD888587028449
:102E200070BD0000002C01400034014070B500224C
:102E300000230024058C4EF6FF7635400584038C74
:102E40008488828B48F6FF752A404FF6FF452A405A
:102E50000D884FF6FF7606EA05252A434DF6FF75E5
:102E60002B400D8906EA05352B434D8806EA0535CA
:102E70002B430B4DA84202D00A4DA84208D14BF675
:102E8000FF752C408D894FF6FF7606EA85152C4399
:102E900084808283CD88A0F84050038470BD0000F8
:102EA000002C0140003401400A460021818B4FF282
:102EB000FF7319404FF6FF7303EA0223194381831E
:102EC00070470021018041808180C1800181418162
:102ED0008181C181704781867047018770478187F2
:102EE0007047A0F840107047002202881D4B98429E
:102EF0000ED01D4B98420BD0B0F1804F08D01B4B29
:102F0000984205D01A4B984202D01A4B984204D1ED
:102F10004FF68F731A404B881A43174B984207D0CD
:102F2000164B984204D04FF6FF431A40CB881A4301
:102F300002808B8883850B8803850A4B98420BD0CF
:102F4000094B984208D00E4B984205D00D4B984241
:102F500002D00D4B984201D10B7A03860123838264
:102F600070470000002C0140003401400004004084
:102F700000080040000C0040001000400014004019
:102F800000400140004401400048014030B589B094
:102F900005460C4601210220FEF77CFA012108209B
:102FA000FEF788FA18208DF823000120ADF82000E4
:102FB00003208DF8220008A91648FDF79AFE00208C
:102FC000ADF81A00ADF81600A8B2ADF81800A0B21E
:102FD000ADF8140000208DF81C0005A90E48FFF77D
:102FE00083FF01A8FFF76DFF6020ADF8040000200B
:102FF000ADF80C000120ADF806000020ADF80A0085
:1030000001A90548FFF7C2FE01210348FFF7E1FDD2
:1030100009B030BD000C01400004004010B540F282
:1030200025510B4800F0DBF880B1094800F092F917
:10303000C4B208480078802808DA074805490978AA
:10304000445404480078401C0249087010BD000038
:1030500000380140BA000020E006002010B540F220
:1030600025511D4800F0BBF810B31B4800F072F961
:10307000C4B21A48008800F40040C8B91748008854
:1030800000F4804060B10A2C03D00020134908806E
:1030900020E01248008840F400401049088019E000
:1030A0000D2C06D10D48008840F480400B49088063
:1030B00010E00A480088C0F30D0009490C54074885
:1030C0000088401C0549088008460088FE2801DD6C
:1030D0000020088010BD000000440040DC000020FB
:1030E000B007002010B586B0044601214804FEF761
:1030F000D1F901210C20FEF7DDF94FF40070ADF895
:10310000140003208DF8160010208DF8170005A973
:103110002248FDF7EEFD0420ADF8140003208DF8E1
:10312000160018208DF8170005A91D48FDF7E1FDD0
:103130000820ADF8140004208DF8170005A91848E0
:10314000FDF7D7FD26208DF8000004208DF8010042
:1031500001208DF803006846FDF730FF0194002040
:10316000ADF80800ADF80A00ADF80C00ADF810009D
:103170000C20ADF80E0001A90A4800F07FF80122EA
:1031800040F22551074800F054F80121054800F0AD
:103190000DF800200449086006B010BD000C014085
:1031A0000008014000440040A481214221B18289ED
:1031B00042F40052828104E082894DF6FF731A4086
:1031C0008281704702460020B1F5007F00D100BF28
:1031D00013880B400BB1012000E00020704770B550
:1031E0000246002400230025002040F66A16B14262
:1031F00000D100BFC1F3421501F01F03012606FAFA
:1032000003F3012D02D19689334006E0022D02D14D
:10321000168A334001E0968A33400C12012606FAE2
:1032200004F41688344013B10CB1012000E00020F2
:1032300070BDF0B50346002400260025002040F6AE
:103240006A17B94200D100BF1846C1F3421401F019
:103250001F06012707FA06F5012C01D10C3004E006
:10326000022C01D1103000E014301AB107682F434E
:10327000076002E00768AF430760F0BD2DE9F04743
:1032800086B005460E460024A24600BFA146002790
:10329000B08900B100BF2F462C8A4CF6FF70044065
:1032A000F08804432C82AC894EF6F3100440B088B9
:1032B00031890843718908430443AC81AC8A4FF6D5
:1032C000FF400440B0890443AC8201A8FEF718F91E
:1032D0001F48874202D1DDF810A001E0DDF80CA004
:1032E000A88900F4004040B10AEBCA0000EB0A10C4
:1032F00031684900B0FBF1F807E00AEBCA0000EBC7
:103300000A1031688900B0FBF1F86420B8FBF0F0D6
:1033100004012009642101FB1089A88900F4004000
:1033200040B1322000EBC900B0FBF1F000F0070023
:10333000044308E0322000EB09106421B0FBF1F0F7
:1033400000F00F0004432C8106B0BDE8F0870000B8
:103350000038014001468888C0F308007047C1F377
:1033600008028280704700BFFEE7000010B50446E7
:10337000240300F0B3F800F0A7F800200B49086020
:103380002020FEF751FFC4F30740FEF74DFFC4F3C2
:103390000720FEF749FFE0B2FEF746FF012004498F
:1033A000C1F8900100F090F810BD0000900121429A
:1033B0000000214208B501210420FEF77BF810200F
:1033C000ADF800008DF8030003208DF80200694677
:1033D0000948FDF78EFC10210748FDF717FD012075
:1033E00006490860FEF7D8FE0020FEF747FF00F010
:1033F00031F80349088008BD0008014090012142CE
:10340000140000202DE9F04106460C461746002026
:103410000F4908600320FEF707FFC4F30740FEF7DB
:1034200003FFC4F30720FEF7FFFEE0B2FEF7FCFE49
:10343000002505E0FF20FEF7F7FE7055681C85B2F9
:10344000BD42F7DB012002490860BDE8F0810000C1
:103450009001214210B5002400200E490860902000
:10346000FEF7E2FE0020FEF7DFFE0020FEF7DCFEA6
:103470000020FEF7D9FEFF20FEF7D6FE44EA002426
:10348000FF20FEF7D1FE044301200349C1F890015B
:10349000204610BD900121420000214210B50024B9
:1034A0000020074908600520FEF7BEFEFF20FEF75A
:1034B000BBFE044601200349C1F89001204610BD1F
:1034C000900121420000214210B500BFFFF7E6FF46
:1034D00000F001000028F9D110BD000010B5002057
:1034E000044908600620FEF79FFE01200249C1F84A
:1034F000900110BD90012142000021422DE9F041D0
:1035000007460E461446F0B2C0F58075AC4200DCAA
:10351000254612E02A463146384600F013F8AC4200
:1035200000D10BE02F442E44601B84B2B4F5807FA1
:1035300002DD4FF4807500E02546EBE700BFBDE8F3
:10354000F08100002DE9F04106460C461746FFF7D2
:10355000C5FF00200F4908600220FEF765FEC4F396
:103560000740FEF761FEC4F30720FEF75DFEE0B200
:10357000FEF75AFE002504E0705DFEF755FE681C5C
:1035800085B2BD42F8DB012002490860FFF79CFFCD
:10359000BDE8F0819001214210B5FFF70BFF00203C
:1035A000FFF7E4FE962000F089FC6C22002107481A
:1035B000FFF7A4FF01226D210548FFF79FFF6C2252
:1035C00000210448FFF71EFF10BD00001C00002072
:1035D00076050020F40500200FB4054B10B503A9B3
:1035E000044A029800F0DAF810BC5DF814FB000001
:1035F0005D3F0008F005002002E008C8121F08C166
:10360000002AFAD170477047002001E001C1121F63
:10361000002AFBD1704700002DE9FF5F82B0002136
:10362000DDE90430020DDDF840B0034318D044F664
:103630001050A2F2FF3242431514119801281FD0F6
:10364000A5EB0B00401C5FEA000A4FF000064E4F4E
:10365000DFF83891B046504615D5CAF1000413E0A2
:10366000119801244AA3012801D16FEA0B010298A5
:10367000119AC0E90031C0E9024206B0BDE8F09FEE
:10368000CBF10000DFE704460021404A491842EB35
:103690000450CDE9001012E0E00707D032463B4667
:1036A00040464946FCF70DFF8046894632463B4678
:1036B00010461946FCF705FF06460F466410002C1D
:1036C000EAD1DDE90401DDE90023BAF1000F06DAF1
:1036D000FCF7F7FE42464B46FCF7F3FE05E0FCF72D
:1036E00062FF42464B46FCF75EFF04460E46002250
:1036F000284BFDF71BF803D84FF0FF30014607E0D9
:103700000022254B20463146FCF734FEFDF762F9D6
:10371000102409E0002C0ADB0A220023FDF764F8DC
:10372000039B30321A55641E50EA0102F2D1641C28
:10373000039AC4F111031444119A012A03D00122FF
:1037400008430DD10AE0084304D000204FF0110BCC
:10375000119072E7A3EB0B056D1E0DE05B4504DDD8
:103760004FF0000205F1010504E003DA4FF000021A
:10377000A5F10105002AECD002981199C0E90231A7
:10378000C0E9004579E70000000014400000F03F68
:10379000300000000000F0430000E03F2DE9FF4F43
:1037A00095B09A46884606460025EEE1252877D151
:1037B00000242746F94A0121039400E0044316F847
:1037C000013F203B01FA03F01042F7D130782A285C
:1037D00011D06FF02F033078A0F13002092A16D8EB
:1037E000039A44F0020402EB820203EB420210440B
:1037F000761C0390EFE758F8042B0392002A03DAB3
:10380000504244F40054039044F00204761C307893
:103810002E2816D116F8010F44F004042A280DD0E2
:103820006FF02F023078A0F13003092B09D807EB95
:10383000870302EB4303C718761CF3E758F8047BB1
:10384000761C30786C280FD006DC4C2817D06828FE
:103850000DD06A2814D104E0742810D07A280FD132
:103860000DE044F400140AE044F4801401E044F450
:1038700040147278824202D104F58014761C761CC2
:10388000307866280BD013DC582877D009DC002864
:1038900075D04528F6D04628F4D047281AD193E1B0
:1038A00018E0632835D0642879D0652812D18BE1DF
:1038B000702873D008DC6728F1D069286FD06E2893
:1038C0000DD06F2806D1ACE073282CD0752874D0A9
:1038D000782853D05246179990476D1C54E1C4F391
:1038E0000250022809D003280DD0D8F8001004286F
:1038F0000DD00D6008F1040846E1D8F80010EA1771
:10390000C1E90052F6E7D8F800100D80F2E70D701B
:10391000F0E718F8041B8DF8001000208DF8010066
:10392000EB46012003E058F804BB4FF0FF3061077D
:103930004FF0000102D40DE009F101018946B942BE
:103940000FDA8145F8DB1BF809100029F4D108E0F3
:1039500009F1010189468142FADB1BF809100029AF
:10396000F6D103985346A0EB090721463846179A2B
:1039700000F080FA284400EB090507E044E008E184
:103980000DE01BF8010B524617999047B9F1010958
:10399000F7D2534621463846179AF2E039E00A2119
:1039A000C4F302524FF0000B0091022A06D058F8DF
:1039B000040BC117032A09D00AE023E008F107002D
:1039C00020F00702F2E80201904605E000B2C117BC
:1039D000042A01D140B2C117002906DA0A460021A3
:1039E000404261EB02012D2202E0220504D52B2288
:1039F0008DF80420012203E0E20701D02022F7E73E
:103A0000914657E00A2100E010214FF0000B009191
:103A10000BE010214FF0000B44F004040827009144
:103A200003E008204FF0000B0090C4F30252022A7A
:103A300005D058F8040B0021032A08D008E008F14B
:103A4000070020F00702F2E80201904603E080B28E
:103A5000042A00D1C0B24FF0000922072AD53278DB
:103A6000702A07D0DDF800C08CF0100C5CEA0B0C5B
:103A700005D00EE040228DF80420012208E050EA33
:103A8000010306D030238DF804308DF80520022282
:103A90009146009B83F0080353EA0B030AD150EAD6
:103AA000010201D1620705D530228DF804204FF0C4
:103AB00001097F1E3278582A04D039A20C920CAA30
:103AC00002920BE03BA2F9E75B46009AFCF78CFE02
:103AD0000C9B9B5C029A521E0292137050EA0102E8
:103AE000F2D1029804A9081A00F1200B600702D550
:103AF00024F4803400E001275F4502DDA7EB0B00D2
:103B000000E0002000EB0B01009003984944401AAC
:103B10000390E00306D453462146179A039800F019
:103B2000A9F90544002706E001A85246C05D17998F
:103B300090476D1C7F1C4F45F6DBE0030CD55346C8
:103B40002146179A039800F095F9054404E03020C7
:103B50005246179990476D1C0099481E0090002905
:103B6000F5DC08E00298029952460078491C02915F
:103B7000179990476D1CBBF10001ABF1010BF1DC13
:103B80005BE100F065F90544761C307800287FF48D
:103B90000DAE19B02846BDE8F08F000009280100DD
:103BA00030313233343536373839616263646566B3
:103BB0000000000030313233343536373839414275
:103BC0004344454600000000600700D4062708F182
:103BD000070020F00700F0E80223804603F0004CC5
:103BE0005FEA0C0001D097A009E0200501D596A05E
:103BF00005E0E00701D095A001E0AFF24C00139082
:103C0000307823F0004365280CD006DC452809D025
:103C100046281DD047287FD13BE0662818D067286A
:103C20007AD136E00021112F01DB112000E0781C51
:103C3000CDE9000104A90CA8FFF7EEFCDDE90D01B8
:103C40000C9A4FF0000B07F10109109200914EE021
:103C50004FF000400097CDE9011004A90CA8FFF730
:103C6000DBFCDDE90D020C9B0F994FF0000B914638
:103C70001093009211B9791C00EB0109B7EB090010
:103C800003D4C0F1FF3B07F10109A9EB0700019044
:103C900042E0012F00DA01270021112F01DD112060
:103CA00000E03846CDE9000104A90CA8FFF7B4FCF8
:103CB000DDE90D010C9A00914FF0000BB94610920E
:103CC00021070FD4009A4A4503DA914601E0A9F191
:103CD0000109B9F1010F05DD109AA9F10101515C4B
:103CE0003029F4D0B84202DA10F1040F03DA0121CE
:103CF000CDE9011010E0002803DC8344A9EB0001AA
:103D000002E0411C494500DD8946A0EB0B00401C48
:103D100001904FF000400290200705D401984845DB
:103D200002DB4FF0FF30019000208DF84B0002982D
:103D30000DF14B07B0F1004F25D002200C902B2045
:103D40000D90029800280CDA404202902D200D9030
:103D500007E00A210298FCF731FD3031029007F8A4
:103D6000011D0C99481E0C900029F2DC02980028D5
:103D7000EFD1791E0D980870307800F0200040F0E7
:103D8000450007F8020D11A8C01BC01D0290139832
:103D9000007800B1012000EB0901019801EBE0710E
:103DA000029801440398401A401E0390E00306D491
:103DB00053462146179A039800F05CF8054413987F
:103DC000007818B15246179990476D1CE00323D52F
:103DD00053462146179A039800F04CF805441BE01F
:103DE000BBF1000F07DB0098584504DD10981799C8
:103DF00010F80B0001E017993020524690470198C7
:103E00000BF1010B401E05F10105019004D12E209C
:103E10005246179990476D1CB9F10001A9F10109AB
:103E2000DEDC05E017F8010B5246179990476D1C30
:103E30000299481E02900029F4DC53462146179A45
:103E400003989EE62D0000002B00000020000000DB
:103E50002DE9F041044600251E461746880404D487
:103E600005E039462020B0476D1C641EF9D5284670
:103E7000BDE8F0812DE9F041044600251E4690463C
:103E8000C80301D5302700E02027880404D505E0C9
:103E900041463846B0476D1C641EF9D52846BDE83A
:103EA000F08170B504460025104603E00E5C6655AF
:103EB0006D1C401C9842F9DB70BD000070B50446D3
:103EC00001F0EEFF012810D00B480088844206D391
:103ED00009480088B4FBF0F5284601F065F906486A
:103EE0000088B4FBF0F100FB11444FF47A7104FB3D
:103EF00001F000F003F870BDDA00002070B5034651
:103F000000224FF0E02675690D4E367803FB06F46B
:103F10004FF0E026B16910E04FF0E026B06988422A
:103F20000BD0884202D20E1A324402E02E1A0E44FE
:103F300032440146A24200D300E0EDE700BF70BD6D
:103F4000D800002030B50446002504E04FF47A7014
:103F5000FFF7D4FF6D1CA542F8D330BD70B5044601
:103F60000D46012008490860E1B20848FFF7F7F95B
:103F700000BF80210548FFF725F90028F9D000206F
:103F800001490860204670BDA481214200440040E0
:103F900002460B46002104E0505C08B10020704747
:103FA000491C9942F8DB0120F9E770B505460C463B
:103FB00045F25550FCF7DCFF2846FCF7CDFF2046C4
:103FC000FCF7D0FFFCF7C0FFFCF7B2FF70BD4FF469
:103FD0004070FDF72BF84820FEF7FEFC4FF416600A
:103FE000FFF780F8FDF738F940F2671140F28F10C3
:103FF000FEF7CCFF4FF49650FDF758FBFCF726FF79
:10400000FDF708FFFEF758FDFEF78CF840F2CF21D0
:1040100040F2F310FDF732F940F2CF2140F2F310F5
:10402000FDF77EF940F2CF2140F2F310FDF7CAF917
:1040300041F61F4142F20F70FEF790FD4FF47A51A6
:104040000520FFF7B2FF0020FDF702FA0020FDF780
:1040500009FA0020FDF70EFA00F002F800BFFEE7B3
:104060001CB5064800210B468022CDE9001004A1B2
:10407000064801F0E5FE01F033FA1CBD680500209A
:1040800073746172745F7461736B0000114D00088A
:104090002DE9F04105460E461C4807681C4800689B
:1040A000001D00F0C3FE50B91948006890F82C10AC
:1040B0000120884017490968814316480160681C3F
:1040C00038B936B112480168091D134800F0ECFEFA
:1040D0001AE07C190E4800684460BC4207D20C48C4
:1040E0000168091D0D48006800F0C4FE0CE0084896
:1040F0000168091D0A48006800F0BCFE0948006814
:10410000844201D207480460BDE8F0810801002024
:10411000F40000200C010020800B0020FC00002097
:10412000F80000202401002010B5044600F0C8FE6D
:1041300023480068401C224908602248006840B9B2
:10414000204804600846006801280DD100F0E4F919
:104150000AE01D48006838B91A480068C06AE16A78
:10416000884201D81748046018480068401C174965
:10417000086094F82C10012088401549096808430C
:1041800013490860E16A01EB8101124A02EB8100E8
:10419000211D00F089FE00F0D7FE0B48006868B1D1
:1041A00008480068C06AE16A884207D24FF0805030
:1041B00009490860BFF34F8FBFF36F8F10BD000038
:1041C00004010020F4000020100100202001002044
:1041D0000C010020B008002004ED00E010B500F054
:1041E0006FFE10480068D0B90F4800F033FE0F484A
:1041F00000F030FE0C480E4908600C480D4908607C
:1042000000220C210A2001F087FA064908600846BE
:10421000006820B108A10348006800F089FF00F0A1
:1042200093FE10BD38010020940B0020A80B002045
:104230003001002034010020546D72510000000054
:1042400070B523E001F0A2F91348006808B9012015
:1042500000E00020054601F0AFFFBDB900F030FEE0
:104260000D48C068C468201D00F0E0FD0B480068E0
:10427000401E0A4908600A480068401E0849086054
:1042800000F062FE204600F060F800BF04480068BD
:104290000028D7D170BD00006C0B00200401002065
:1042A0000001002070B504460D46206C70B1216CF1
:1042B000E0680844E0606168E068884201D32068F3
:1042C000E0602846226CE168FBF77AFF70BD2DE9BB
:1042D000F04104460F4615464FF00008A66B206CCF
:1042E00040B9206860BB606801F0A0FE80460020F5
:1042F000606025E07DB93946226CA068FBF760FF5D
:10430000216CA0680844A060D4E90110884217D34A
:104310002068A06014E03946226CE068FBF750FF8B
:10432000216CE068401AE0602168E068884203D2AE
:10433000216C6068401AE060022D01D106B1761E42
:10434000701CA0634046BDE8F08110B50446206BA8
:1043500000F032FE204600F02FFE10BD0146084A54
:10436000126812680AB9012200E000220A600A6895
:1043700022B9034A1268D268106800E00020704732
:104380003001002030B54FF42053174800F00704E7
:104390002CB1C01D20F00700134C041B1B1B024650
:1043A000124C22600024114D6C60D018083820F0A7
:1043B00007000F4C206000240D4D2D686C600C4DE3
:1043C0002D682C601146441A4C60094C24680C601E
:1043D000084D4C682C60084D4C682C604FF0004430
:1043E000064D2C6030BD00000C0C00205001002058
:1043F00058010020600100205C01002064010020C1
:1044000000BFFFF71DFF064800680128F9D94FF0EB
:10441000805004490860BFF34F8FBFF36F8FF0E700
:10442000B008002004ED00E02DE9F04106460D46FD
:1044300017469846069C0DB9246000E02760E663A5
:1044400025640121204601F0ADFA0020A064BDE8FA
:10445000F08100002DE9FF5F81460F469246DDE9BD
:104460000E6B109CAAF10100216B01EB800828F073
:10447000070808F0070008B9012000E0002028B96B
:1044800040F22B321BA120A0FFF7A6F8002507E081
:10449000795D04F134004155785D00B902E06D1C8E
:1044A000102DF5D300BF002143200155202E00D34D
:1044B0001F26E66266640020A064201D00F0D7FC81
:1044C00004F1180000F0D3FC2461C6F12000A061C3
:1044D00064620020E06484F8500049464046039A34
:1044E00000F004FC2060BBF1000F01D0CBF80040CD
:1044F000BDE8FF9F2E2E5C4672656552544F535C9B
:104500007461736B732E63004572726F723A257318
:104510002C25640D0A00000010B5002407E004EB10
:1045200084010F4A02EB810000F094FC641C202CF3
:10453000F5D30C4800F08EFC0B4800F08BFC0B48C8
:1045400000F088FC0A4800F085FC0A4800F082FC74
:1045500004480949086004480849086010BD000083
:10456000B0080020300B0020440B0020580B002026
:104570006C0B0020800B0020F8000020FC000020C5
:1045800010B50146164800E0006803688B42FBD373
:104590000246436813448B4204D143684C68234469
:1045A000436001460A464B6813440468A34211D194
:1045B0000C4C03682468A34208D04B680468646804
:1045C00023444B6003681B680B6005E0054B1B68C8
:1045D0000B6001E003680B60884200D0016010BDF1
:1045E00050010020580100202DE9F04104460D46FD
:1045F00016461F464FF0000865602461B5420CD88E
:10460000F01BA169884202D34FF0010811E0211D7F
:104610000948006800F02EFC0BE0BE4204D2BD4207
:1046200002D34FF0010804E0211D0448006800F0A7
:1046300021FC4046BDE8F08134010020300100201B
:1046400070B5054600F03CFCA86B08B9012400E0F9
:10465000002400F079FC204670BD70B5054600F0DE
:104660002FFCA86BE96B884201D1012400E00024F3
:1046700000F06AFC204670BD2DE9F3410D4600981C
:10468000846C00272CB940F6CE121AA128A0FEF7A0
:10469000A3FFA06BE16B884201D2012000E0002063
:1046A00028B940F6CF1213A121A0FEF795FFA06B09
:1046B000E16B88421BD294F945602A466946204640
:1046C000FFF705FE0746701C60B9606A08B9012053
:1046D00000E0002050B904F1240001F013FD28B1DE
:1046E000012703E0701C40B284F8450000BF384643
:1046F000BDE8FC812E2E5C2E2E5C2E2E5C73746D1C
:1047000033322D636F6E74726F6C205F6C69616EF3
:1047100077616E675C636F6E74726F6C5C46726516
:104720006552544F535C71756575652E63000000CA
:104730004572726F723A25732C25640D0A000000D1
:10474000F8B505460F4613480068C068C468201DC8
:1047500000F06CFBE069012818D1A06941192B46D3
:104760003A462046FFF740FF80B1002003462A4624
:1047700001460090204601F0E9FD06462EB94FF4AF
:10478000027205A10AA0FEF727FF00BF2046616A5A
:104790008847F8BD300100202E2E5C4672656552B8
:1047A000544F535C74696D6572732E630000000092
:1047B0004572726F723A25732C25640D0A00000051
:1047C00070B586B060E0039800285DDB059C6069E9
:1047D00008B9012000E0002010B9201D00F026FBE0
:1047E00002A800F0C7F8054603980A284AD2DFE875
:1047F00000F00905072C2E4506082D2F00BF00BF2D
:1048000000BF00BF0498A269811803462A462046CB
:10481000FFF7EAFEC0B12046616A8847E0690128D7
:1048200012D1002000900498A16942180023194673
:10483000204601F08BFD06462EB940F2213218A128
:104840001DA0FEF7C9FE00BF1DE000BF1BE000BFBA
:104850000498A061A06908B1012000E0002028B9F7
:104860004FF44E720EA114A0FEF7B6FEA0694119D6
:104870002B462A462046FFF7B7FE04E0204600F00C
:104880009BFB00E000BF00BF00231A4603A90E48AF
:10489000006800F08FFF002895D106B070BD0000C1
:1048A0002E2E5C4672656552544F535C74696D657B
:1048B00072732E63000000004572726F723A2573A6
:1048C0002C25640D0A00000038010020F8B50546CB
:1048D0000C4600F05BFE684600F04CF80646009877
:1048E00020BB44B9B54206D801F066FC31462846E3
:1048F000FFF726FF1CE03CB10E480068006808B9CD
:10490000012000E000200446A91B22460A48006856
:1049100000F024FC01F050FC50B94FF080500749E2
:104920000860BFF34F8FBFF36F8F01E001F044FCCD
:10493000F8BD0000340100203801002004ED00E043
:104940000A490968096809B9012100E0002121B17B
:104950004FF0FF31064A116006E004490968C96852
:10496000C868034A4168116070470000F8000020E1
:104970002401002070B5044601F0A2FA054607485C
:104980000068854204D200F00BF80120206001E0AD
:104990000020206001480560284670BD40010020CD
:1049A0002DE9F8432DE021480068C06805681F48DC
:1049B0000068C068C468201D00F038FA2046616AAB
:1049C0008847E06901281CD1A0694619AE4207D981
:1049D00066602461211D1548006800F04BFA10E064
:1049E000002003462A4601460090204601F0AEFC16
:1049F00007462FB940F292320DA113A0FEF7ECFD4D
:104A000000BF0A480068006808B9012000E00020E3
:104A10000028C8D00548D0F800800F480068034936
:104A200008600D48C0F80080BDE8F8833001002020
:104A30002E2E5C4672656552544F535C74696D65E9
:104A400072732E63000000004572726F723A257314
:104A50002C25640D0A000000340100200B4800687A
:104A6000401C08B9012000E0002020B9F42208A170
:104A700012A0FEF7B1FD00BF502080F31188BFF3F4
:104A80004F8FBFF36F8F00BF00BFFEE744010020D0
:104A90002E2E5C4672656552544F535C706F727473
:104AA00061626C655C525644535C41524D5F434DAC
:104AB000335C706F72742E63000000004572726F79
:104AC000723A25732C25640D0A00000008B500BF5A
:104AD0006846FFF743FC044620460099FFF7F6FEC0
:104AE000FFF76EFEF4E770B5044600F0E9F994F9BB
:104AF00045501AE0A06C38B100212046FFF7BCFDFC
:104B000088B100F011FC0EE0606A08B9012000E0F5
:104B1000002038B904F1240001F0F4FA18B100F0D3
:104B200003FC00E003E0681E45B2002DE2DC00BF9C
:104B3000FF2084F8450000F007FA00F0C1F994F96D
:104B4000445010E0206908B9012000E0002048B975
:104B500004F1100001F0D6FA08B100F0E5FB681E80
:104B600045B200E001E0002DECDC00BFFF2084F83E
:104B7000440000F0E9F970BD2DE9F04104464FF022
:104B8000000800F003FD3E48006808B9FFF7FAFB93
:104B90003C480068204000285FD1A4B1083404F0EC
:104BA000070080B104F00700C0F10800044404F0DD
:104BB000070008B9012000E0002020B9BF2232A17F
:104BC0003BA0FEF709FD002C47D03D480068844219
:104BD00043D83C4E3046056801E02E462D68686893
:104BE000A04202D228680028F7D1254800688542F3
:104BF00033D0306800F10808286830606868001B0E
:104C0000102813D92F1907F0070008B9012000E078
:104C1000002020B9EC221CA125A0FEF7DDFC68686D
:104C2000001B78606C603846FFF7AAFC244968686E
:104C30000968081A2249086008460068224909687C
:104C4000884203D21E4800681F4908600D49686801
:104C50000968084368600020286001F0ADFA08F098
:104C6000070008B9012000E0002028B94FF496722F
:104C700005A10FA0FEF7B0FC4046BDE8F0810000A2
:104C800058010020640100202E2E5C46726565529A
:104C9000544F535C706F727461626C655C4D656DEE
:104CA0004D616E675C686561705F342E6300000063
:104CB0004572726F723A25732C25640D0A0000004C
:104CC0005C010020500100206001002006480068BF
:104CD00030B10549096801F14800896C491C01603F
:104CE0000148006870470000F4000020001F4FF0EA
:104CF00080730360001F21F001030360001F034B5A
:104D00000360143802602038704700005D4A0008D4
:104D10001CB5044600F0D4F80948012100234A02DA
:104D2000CDE9001007A10E4801F08AF80D4908608E
:104D30000D48006800F072FA00F006F91CBD000092
:104D40006C05002053656E736F725F436F6D6D75F8
:104D50006E69636174696F6E5F7461736B000000EC
:104D600019230008C0050020680500201CB528494B
:104D70002848FCF73DFF27480078C0EB0010244985
:104D8000097801EB8000244908802448007800EB72
:104D9000C00040000E382249095C2048007800EB32
:104DA000C00040000F381E4A105CC0EB001001EB41
:104DB00080001C490880184800880988884220DB48
:104DC00000200090034601220921019040F2E77083
:104DD000FDF732F911480078062806D10120124962
:104DE0000870FEF7D9FB01201CBD0C480078401C60
:104DF0000D490870FEF7D0FB08480078401CC0B28F
:104E0000F2E7064800780849087004480078EBE7A4
:104E10008305002082050020180000208B0500205B
:104E20001C0000201A0000207605002001460A69B7
:104E3000D1E901309860D1E9010358605068884297
:104E400001D188685060002008611068401E106021
:104E50001068704700F1080141604FF0FF31816038
:104E600000F10801C160016100210160704700216B
:104E70000161704710B502460B685C1C0CB91069E3
:104E800007E002F1080000E04068446824689C42A2
:104E9000FAD944684C604C68A160886041600A613E
:104EA0001468641C146010BD42684A6093688B608B
:104EB000936859609160086103685B1C03607047E8
:104EC00010B500BF502080F31188BFF34F8FBFF3A0
:104ED0006F8F00BF0B480068401C0A4908600846F5
:104EE000006801280DD108480068C0B208B9012047
:104EF00000E0002028B94FF4BD7204A10EA0FEF717
:104F00006BFB10BD4401002004ED00E02E2E5C463A
:104F100072656552544F535C706F727461626C6558
:104F20005C525644535C41524D5F434D335C706F4D
:104F300072742E63000000004572726F723A25731E
:104F40002C25640D0A00000010B50B48006828B934
:104F500040F2811209A114A0FEF73EFB064800684A
:104F6000401E054908600846006820B9002080F30B
:104F7000118800BF00BF10BD440100202E2E5C46EA
:104F800072656552544F535C706F727461626C65E8
:104F90005C525644535C41524D5F434D335C706FDD
:104FA00072742E63000000004572726F723A2573AE
:104FB0002C25640D0A00000070B506463546002E0B
:104FC00035D0083D2C461A4960680968084008B188
:104FD000012000E0002028B94FF4A07215A11FA005
:104FE000FEF7FAFA206808B9012000E0002028B98D
:104FF00040F241120FA119A0FEF7EEFA0C496068C9
:105000000968084098B1206888B90949606809684A
:105010008843606000F0BAFA14496068096808447F
:10502000124908602046FFF7ABFA01F0C5F870BDE1
:10503000640100202E2E5C4672656552544F535C0D
:10504000706F727461626C655C4D656D4D616E6709
:105050005C686561705F342E630000004572726F9A
:10506000723A25732C25640D0A0000005C010020B3
:10507000064800684FF47A71B0FBF1F0401E4FF023
:10508000E02148610720086170470000000000200F
:1050900070B5FBF77FF80546102D11D305F1E02020
:1050A00090F8F04310480078844201DB012000E0D2
:1050B000002028B94FF42A720CA117A0FEF78CFA31
:1050C0001948006800F4E06018490968884201D86E
:1050D000012000E0002028B94FF42E7203A10EA099
:1050E000FEF77AFA70BD0000480100202E2E5C46C3
:1050F00072656552544F535C706F727461626C6577
:105100005C525644535C41524D5F434D335C706F6B
:1051100072742E63000000004572726F723A25733C
:105120002C25640D0A0000000CED00E04C0100206D
:10513000024600200BE0084B53F8303033B9064BE1
:1051400043F8301003EBC0035A6002E0401C0A2809
:10515000F1D300BF70470000BC0B00202DE9F041E7
:1051600005460E4617462C46FFF7AAFE94F9440062
:10517000401C10B9002084F8440094F94500401CFC
:1051800010B9002084F84500FFF7DEFEA06B28B9B7
:105190003A46314604F1240000F0F6F82046FFF7C5
:1051A000A2FCBDE8F081000070B504460025ACB15A
:1051B0000F48006808B9012000E0002028B940F23B
:1051C000CF420CA110A0FEF707FA00F0DFF9002192
:1051D0002046FEF75DFF00F0EFFF05463DB94FF0BA
:1051E00080500D490860BFF34F8FBFF36F8F70BDC4
:1051F0002C0100202E2E5C4672656552544F535C84
:105200007461736B732E63004572726F723A25730B
:105210002C25640D0A00000004ED00E070B5054681
:10522000FFF74EFE15B92D48006800E028460446F9
:10523000201DFFF7FBFD78B9E06A00EB80002849EC
:1052400051F8200040B994F82C10012088402549DD
:105250000968814323480160A06A18B104F118006D
:10526000FFF7E4FD20480068401C1F4908601B4808
:105270000068844209D1211D1C48FFF715FE1C4817
:105280000068401C1A49086009E01A480068401E7E
:10529000184908602046FFF758F8FFF751FBFFF761
:1052A00053FE15480068C0B10C480068844214D110
:1052B0001248006808B9012000E0002028B940F237
:1052C00065420FA113A0FEF787F94FF080501549F2
:1052D0000860BFF34F8FBFF36F8F70BDF4000020E5
:1052E000B00800200C010020200100206C0B0020E1
:1052F0000001002004010020100100202C010020EA
:105300002E2E5C4672656552544F535C7461736B0C
:10531000732E63004572726F723A25732C25640DEB
:105320000A00000004ED00E0012001490860704718
:105330001801002070B504460D462CB940F606321F
:1053400007A10CA0FEF748F90E4801681831204665
:10535000FFF790FD01212846FEF79AFE70BD000080
:105360002E2E5C4672656552544F535C7461736BAC
:10537000732E63004572726F723A25732C25640D8B
:105380000A000000F400002070B505460E461446E1
:105390002DB940F6313209A10DA0FEF71DF91048D4
:1053A000016818312846FFF77FFD0CB14FF0FF363A
:1053B00021463046FEF76CFE70BD00002E2E5C4686
:1053C00072656552544F535C7461736B732E630046
:1053D0004572726F723A25732C25640D0A00000025
:1053E000F400002070B505462C46002D4BD0264910
:1053F000E06A0968C96A884245D2A06900F00040A5
:1054000028B921480068C06AC0F12000A061E16AA3
:1054100001EB81011D4A02EB81016069884201D1E3
:10542000012000E0002050B3201DFFF7FFFC78B9F9
:10543000E06A00EB8000154951F8200040B994F86B
:105440002C100120884012490968814310480160EE
:105450000D480068C06AE06294F82C100120884072
:105460000B49096808430A490860E16A01EB8101B8
:10547000064A02EB8100211DFFF716FD03E00248FA
:105480000068C06AE06270BDF4000020B00800202F
:105490000C01002010B504462CB940F6C13205A11C
:1054A00009A0FEF799F80C48006820600B480068D6
:1054B000606010BD2E2E5C4672656552544F535C81
:1054C0007461736B732E63004572726F723A257349
:1054D0002C25640D0A0000001C010020080100209A
:1054E0001CB51A4800210B468022CDE9001018A1F6
:1054F000194800F0A5FC0446012C02D100F0ECFE96
:105500000446012C15D100BF502080F31188BFF351
:105510004F8FBFF36F8F00BF4FF0FF300F49086010
:1055200001200F49086000200E49086000F08AF849
:105530000BE0601C08B1012000E0002028B940F217
:10554000847209A10DA0FEF747F81CBD28010020B8
:1055500049444C450000000001440008240100209B
:1055600010010020080100202E2E5C467265655255
:10557000544F535C7461736B732E63004572726F8A
:10558000723A25732C25640D0A0000000248006859
:10559000401C0149086070472C01002010B51B48D1
:1055A000006818B101201A4908602DE00020184950
:1055B000086018480068B0FA80F0C0F11F0404EBDE
:1055C0008400154951F8200008B1012000E00020B6
:1055D00028B940F6F62211A115A0FDF7FDFF04EB56
:1055E00084010D4A02EB810041684968416000F185
:1055F000080142688A4202D14168496841604168B5
:10560000C9680F4A116000BF10BD00002C010020C6
:10561000180100200C010020B00800202E2E5C464E
:1056200072656552544F535C7461736B732E6300E3
:105630004572726F723A25732C25640D0A000000C2
:10564000F40000201CB52248014609780191FF2191
:10565000024611700146097800919DF8001001F092
:1056600050011C4A117007211B4A116009E01A49B8
:105670000968491E184A11609DF800104906090E74
:1056800000919DF8001001F080018029EFD01249AF
:1056900009680902104A11601146098801F4E061A5
:1056A00011600B4A019911700C48006840F47000B9
:1056B0000A4908600846006840F070400860FFF73B
:1056C000D7FC002006490860FAF72EFD00201CBD1B
:1056D00000E400E0480100204C01002020ED00E043
:1056E0004401002010B500BF502080F31188BFF3A3
:1056F0004F8FBFF36F8F00BF00F0E8FB18B14FF082
:1057000080500449086000BF002080F3118800BF6A
:1057100010BD000004ED00E02DE9F84305460E46FB
:1057200090460DB1012000E0002028B94FF4C4726A
:105730000DA11CA0FDF750FF0EB9002701E005FBED
:1057400006F707F14C00FFF717FA044644B104F1DD
:105750004C0943464A46314628460094FEF764FE0B
:105760002046BDE8F88300002E2E5C2E2E5C2E2EE7
:105770005C73746D33322D636F6E74726F6C205F67
:105780006C69616E77616E675C636F6E74726F6C6B
:105790005C4672656552544F535C71756575652E34
:1057A000630000004572726F723A25732C25640DF8
:1057B0000A0000002DE9FF4782B005460E461F464D
:1057C0004FF0000A2C462CB940F2DC4261A170A0D7
:1057D000FDF702FF0EB9206C08B9012000E000209F
:1057E00028B940F2DD425BA169A0FDF7F5FE00F0AB
:1057F00057FB08B9049808B9012000E0002028B937
:105800004FF49C6253A162A0FDF7E6FE00BFFFF7D4
:1058100057FBD4F83890B9F1000F3DD0D4F80C8084
:1058200031462046FEF73EFDDFB9A9F10100A06335
:10583000206810B9FFF74AFA6060206908B90120B2
:1058400000E0002010BB04F1100000F05BFCE8B1A8
:105850004FF0805052490860BFF34F8FBFF36F8FF6
:1058600014E0C4F80C80606A08B9012000E0002050
:1058700060B904F1240000F045FC38B14FF08050CD
:1058800047490860BFF34F8FBFF36F8FFFF75CFB93
:10589000012006B0BDE8F087049818B9FFF754FB63
:1058A0000020F6E7BAF1000F04D16846FFF7F2FDD9
:1058B0004FF0010AFFF748FBFFF768FEFFF700FB18
:1058C00094F94400401C10B9002084F8440094F975
:1058D0004500401C10B9002084F84500FFF734FB58
:1058E00004A9684600F05CFA40BB2046FEF7A8FE1B
:1058F000F0B1206830B9FFF7E3FA6068FFF772FD96
:10590000FFF722FB04F124000499FFF713FD204662
:10591000FFF7E9F800F050FC00287FF478AF4FF073
:1059200080501F490860BFF34F8FBFF36F8F6EE742
:105930002046FFF7D8F800F03FFC68E72046FFF765
:10594000D2F800F039FC2046FEF77AFE0028EED0AF
:1059500000209EE72E2E5C2E2E5C2E2E5C73746D26
:1059600033322D636F6E74726F6C205F6C69616E81
:1059700077616E675C636F6E74726F6C5C467265A4
:105980006552544F535C71756575652E6300000058
:105990004572726F723A25732C25640D0A0000005F
:1059A00004ED00E070B505460E462C462CB940F2D9
:1059B0001B121EA12CA0FDF70FFEFFF781FAD4E900
:1059C0000F12206801FB020060600020A0632068C5
:1059D000A060E06B401E226C216800FB0210E060BA
:1059E000FF2084F8440084F845009EB9206908B976
:1059F000012000E00020A8B904F1100000F082FBB3
:105A000080B14FF080501C490860BFF34F8FBFF347
:105A10006F8F07E004F11000FFF71CFA04F1240077
:105A2000FFF718FAFFF790FA012070BD2E2E5C2EBA
:105A30002E5C2E2E5C73746D33322D636F6E747218
:105A40006F6C205F6C69616E77616E675C636F6E0F
:105A500074726F6C5C4672656552544F535C71751D
:105A60006575652E630000004572726F723A25738A
:105A70002C25640D0A00000004ED00E02DE9FF4331
:105A800083B0064688461D464FF0000934462CB9BF
:105A900040F2D92260A16FA0FDF79EFDB8F1000F82
:105AA00001D1206C08B9012000E0002028B940F2A3
:105AB000DA2259A167A0FDF78FFD022D02D1E06B1C
:105AC000012801D1012000E0002028B940F2DB22AA
:105AD00051A160A0FDF780FD00F0E2F908B905983A
:105AE00008B9012000E0002028B940F2DE224AA1D6
:105AF00058A0FDF771FD00BFFFF7E2F9A06BE16B65
:105B0000884201D3022D38D12A4641462046FEF76D
:105B1000DEFB0746A06C68B129462046FEF7ACFDC7
:105B200028B34FF080504F490860BFF34F8FBFF349
:105B30006F8F1CE0606A08B9012000E0002068B99E
:105B400004F1240000F0DEFA88B14FF0805045499E
:105B50000860BFF34F8FBFF36F8F08E03FB14FF086
:105B6000805040490860BFF34F8FBFF36F8FFFF73E
:105B7000EBF9012007B0BDE8F083059818B9FFF7ED
:105B8000E3F90020F6E7B9F1000F04D101A8FFF70F
:105B900081FC4FF00109FFF7D7F9FFF7F7FCFFF79A
:105BA0008FF994F94400401C10B9002084F8440097
:105BB00094F94500401C10B9002084F84500FFF717
:105BC000C3F905A901A800F0EBF8F0B92046FEF7EB
:105BD00044FDA0B104F110000599FFF7ABFB20468E
:105BE000FEF781FF00F0E8FA002885D14FF08050E1
:105BF0001C490860BFF34F8FBFF36F8F7CE72046CF
:105C0000FEF771FF00F0D8FA76E72046FEF76BFF4B
:105C100000F0D2FA0020ADE72E2E5C2E2E5C2E2E48
:105C20005C73746D33322D636F6E74726F6C205FB2
:105C30006C69616E77616E675C636F6E74726F6CB6
:105C40005C4672656552544F535C71756575652E7F
:105C5000630000004572726F723A25732C25640D43
:105C60000A00000004ED00E02DE9F05F80468A465E
:105C700015461E4644462CB940F29F3235A144A039
:105C8000FDF7AAFCBAF1000F01D1206C08B9012080
:105C900000E0002028B94FF468722EA13CA0FDF767
:105CA0009BFC022E02D1E06B012801D1012000E013
:105CB000002028B940F2A13226A135A0FDF78CFCC6
:105CC000FFF7E6F900BF5021EFF3118081F311884F
:105CD000BFF34F8FBFF36F8F00BF0746A06BE16B21
:105CE000884201D3022E2BD194F945B03246514659
:105CF0002046FEF7ECFA0BF10100C8B9A06C40B1E8
:105D000031462046FEF7B8FCB8B1B5B10120286095
:105D100013E0606A08B9012000E0002068B904F1CE
:105D2000240000F0EFF940B13DB10120286004E00B
:105D30000BF1010040B284F845004FF0010901E089
:105D40004FF0000900BF87F3118800BF4846BDE847
:105D5000F09F00002E2E5C2E2E5C2E2E5C73746D38
:105D600033322D636F6E74726F6C205F6C69616E7D
:105D700077616E675C636F6E74726F6C5C467265A0
:105D80006552544F535C71756575652E6300000054
:105D90004572726F723A25732C25640D0A0000005B
:105DA0002DE9F04104460D462CB940F6CB3219A13D
:105DB0001DA0FDF711FC2DB940F6CC3215A11AA09B
:105DC000FDF70AFCFFF77CF81B4807682868401CB1
:105DD00008B9002619E0194920680968884204D0EA
:105DE0006068B84201D801260FE06068381A296857
:105DF000884209D228686168791A401A28602046CA
:105E0000FFF748FB002600E00126FFF79DF830462B
:105E1000BDE8F0812E2E5C4672656552544F535C8E
:105E20007461736B732E63004572726F723A2573DF
:105E30002C25640D0A000000080100201C01002030
:105E40002DE9FF4F85B0804689461746DDE912AB44
:105E5000B800FEF791FE064656B15420FEF78CFEC0
:105E600004460CB1266304E03046FFF7A5F800E0D5
:105E700000247CB10020CDE900ABCDE902403A46D8
:105E800049464046089BFEF7E5FA2046FEF74CF9E6
:105E9000012501E04FF0FF35284609B0BDE8F08F3D
:105EA0000549096809B9012005E00449096809B9EB
:105EB000022000E000207047100100202C0100208B
:105EC0000149086870470000080100202DE9F041F1
:105ED0004FF0000841480068002872D1404800682F
:105EE000451C3F480560EDB93E480068006808B9A8
:105EF000012000E0002028B940F6D9123AA13FA0C5
:105F0000FDF76AFB37480768404800683549086074
:105F10003E4807603E480068401C3D490860FEF767
:105F20000FFD00BF3B48006885423CD300BF2D48B1
:105F30000068006808B9012000E0002020B14FF09F
:105F4000FF30344908602DE026480068C068C46806
:105F50006668B54202D22F48066023E0201DFEF796
:105F600065FFA06A18B104F11800FEF75FFF94F80E
:105F70002C100120884028490968084326490860F8
:105F8000E16A01EB8101254A02EB8100211DFEF748
:105F90008BFF2349E06A0968C96A8842C7D34FF07A
:105FA0000108C4E700BF1E480068C06A00EB80001B
:105FB0001A4951F82000012801D94FF0010805E0E5
:105FC000FFE718480068401C16490860164800683A
:105FD00008B14FF001084046BDE8F0812C010020D7
:105FE00008010020F80000202E2E5C4672656552E4
:105FF000544F535C7461736B732E63004572726F00
:10600000723A25732C25640D0A000000FC00002064
:106010001C010020240100200C010020B0080020F9
:10602000F4000020140100201801002070B505467E
:106030002C460026002D4BD026480068844201D112
:10604000012000E0002028B940F6C76222A127A065
:10605000FDF7C2FAA06C28B940F6C9621EA123A0C0
:10606000FDF7BAFAA06C401EA064616CE06A884239
:106070002ED0A06C60BB201DFEF7D8FE78B9E06A78
:1060800000EB80001D4951F8200040B994F82C1015
:10609000012088401A490968814319480160606CF1
:1060A000E062E06AC0F12000A06194F82C100120A9
:1060B000884013490968084311490860E16A01EB07
:1060C00081010E4A02EB8100211DFEF7EDFE012643
:1060D000304670BDF40000202E2E5C46726565527D
:1060E000544F535C7461736B732E63004572726F0F
:1060F000723A25732C25640D0A000000B0080020B8
:106100000C01002070B50646F068C4682CB940F652
:1061100061321AA11EA0FDF75FFA04F11800FEF724
:1061200085FE1F480068A8B9201DFEF77FFE94F881
:106130002C10012088401B49096808431949086050
:10614000E16A01EB8101184A02EB8100211DFEF793
:10615000ABFE04E004F118011448FEF7A5FE144953
:10616000E06A0968C96A884204D9012501201149F9
:10617000086000E00025284670BD00002E2E5C4619
:1061800072656552544F535C7461736B732E630078
:106190004572726F723A25732C25640D0A00000057
:1061A0002C0100200C010020B0080020580B00201A
:1061B000F40000201801002070B5002400263448A7
:1061C000006828B94FF4FD6232A137A0FDF704FA48
:1061D000FEF776FE2E480068401E2D4908600846EE
:1061E000006800284FD13448006800284BD024E0D4
:1061F0003248C068C46804F11800FEF717FE201D7D
:10620000FEF714FE94F82C10012088402C490968F0
:1062100008432B490860E16A01EB8101294A02EB3E
:106220008100211DFEF740FE2749E06A0968C96A1E
:10623000884202D30120254908602048006808B937
:10624000012000E000200028D2D00CB1FEF778FB3E
:106250001F48056865B100BFFFF738FE10B1012087
:106260001A4908606D1E002DF6D1002018490860FB
:106270001648006838B10126300716490860BFF398
:106280004F8FBFF36F8FFEF75FFE304670BD00008B
:106290002C0100202E2E5C4672656552544F535CD3
:1062A0007461736B732E63004572726F723A25735B
:1062B0002C25640D0A00000004010020580B00206A
:1062C0000C010020B0080020F4000020180100207C
:1062D0001401002004ED00E01CB50024FDF77EFF52
:1062E0000B48006858B10B481F2100234FF48072FF
:1062F000CDE9001008A10A48FFF7A2FD04462CB919
:1063000040F2331207A10DA0FDF766F920461CBD2F
:10631000380100203C010020546D72205376630048
:10632000CD4A00082E2E5C4672656552544F535C70
:1063300074696D6572732E63000000004572726FA0
:10634000723A25732C25640D0A0000002DE9FE43E6
:1063500004460D4616461F46DDF828804FF000091A
:106360002CB94FF4D37216A11BA0FDF735F91E48C6
:10637000006810B3009501960294062D15DAFFF718
:106380008FFD022808D1002342466946164800685E
:10639000FFF774FB814610E000231A466946124855
:1063A0000068FFF76BFB814607E000233A46694629
:1063B0000D480068FFF758FC81464846BDE8FE835B
:1063C0002E2E5C4672656552544F535C74696D6540
:1063D00072732E63000000004572726F723A25736B
:1063E0002C25640D0A0000003801002000C1814006
:1063F00001C0804101C0804100C1814001C0804195
:1064000000C1814000C1814001C0804101C0804184
:1064100000C1814000C1814001C0804100C1814074
:1064200001C0804101C0804100C1814001C0804164
:1064300000C1814000C1814001C0804100C1814054
:1064400001C0804101C0804100C1814000C1814044
:1064500001C0804101C0804100C1814001C0804134
:1064600000C1814000C1814001C0804101C0804124
:1064700000C1814000C1814001C0804100C1814014
:1064800001C0804101C0804100C1814000C1814004
:1064900001C0804101C0804100C1814001C08041F4
:1064A00000C1814000C1814001C0804100C18140E4
:1064B00001C0804101C0804100C1814001C08041D4
:1064C00000C1814000C1814001C0804101C08041C4
:1064D00000C1814000C1814001C0804100C18140B4
:1064E00001C0804101C0804100C1814000C0C101A4
:1064F000C30302C2C60607C705C5C404CC0C0DCD34
:106500000FCFCE0E0ACACB0BC90908C8D81819D9A3
:106510001BDBDA1A1EDEDF1FDD1D1CDC14D4D515D3
:10652000D71716D6D21213D311D1D010F03031F1C3
:1065300033F3F23236F6F737F53534F43CFCFD3DF3
:10654000FF3F3EFEFA3A3BFB39F9F83828E8E929E3
:10655000EB2B2AEAEE2E2FEF2DEDEC2CE42425E593
:1065600027E7E62622E2E323E12120E0A06061A103
:1065700063A3A26266A6A767A56564A46CACAD6DB3
:10658000AF6F6EAEAA6A6BAB69A9A86878B8B97923
:10659000BB7B7ABABE7E7FBF7DBDBC7CB47475B553
:1065A00077B7B67672B2B373B17170B05090915143
:1065B0009353529296565797559594549C5C5D9D73
:1065C0005F9F9E5E5A9A9B5B995958988848498963
:1065D0004B8B8A4A4E8E8F4F8D4D4C8C4484854513
:1065E00087474686824243834181804000030306F9
:1065F00001040602050003051F1C1F1E1F1E1F1F8E
:106600001E1F1E1F2466000800000020F405000065
:10661000280A0008F8660008F4050020A4330000EA
:10662000083600081184A24A04500C010203040633
:1066300007080917EF011CEEEE011C14FA02BC2A30
:106640006402FFFFFFFFEEEE0212FA0312FA0412D9
:10665000FA0512EA06120316B5050D12FFFCFFFF3C
:1066600017091115256F12833AE3AA4329D669DA6F
:106670000552020406081AAA0101200033FF2F73F5
:1066800079732F6870386F51684D5A4A36372F44E6
:106690006576696365312F7468696E672F65766505
:1066A0006E742F70726F70657274792F706F73745F
:1066B00001CF28232F7379732F6870386F51684D7D
:1066C0005A4A36372F446576696365312F74686995
:1066D0006E672F7365720F180A2F70726F70657274
:1066E00074791102FF7401DCBA0107C91589101A07
:0866F0000313045109D40C004E
:04000005080000ED02
:00000001FF
